:020000040000FA
:10000000B6018E29A4003A0884003808F62084132B
:1000100000052C1C3806031920282408031D182865
:100020002A08FF3E031C212864300A212A082128BF
:10003000240AFF3003192028240B20282B0821280C
:10004000AD09AD0C8929B616B61EB612B6192C2804
:10005000B6156520031853280830A3007920A20D97
:10006000A30B2E28B61E5E2083207F20B61A5320B5
:100070005820220803108929B616B61EB612361962
:100080004628FE39B700361503108929361A4E283E
:10009000A600361665200318532826086C2003187E
:1000A0005328B61E89295E20832036113612B611D8
:1000B0003A08840038088417800464283A088400C9
:1000C00038098005841780050800582083205E20A9
:1000D0007F203708B6190138A2000830A300A20D0E
:1000E00003185820031C5E2083207F20A30B6F2859
:1000F000582083203A08840038080005FF3E3B085A
:100100008400390961283B08840039085B28A5016F
:10011000A400B7172730A30010309A200330A300A3
:10012000E8309A20A30164309A20A3010A309A2073
:100130002408A528A2002508A1002408A000572112
:100140002008031DB713B71B0800303EA700851316
:10015000051305138316851305130513F030850564
:1001600083122708B618D2283A30A10098301821F7
:100170003330A600E7201330A10088301821E72093
:1001800064301721E720643017212230A600E720D1
:100190002830D1200C30D1200630D120B6142708C9
:1001A000D2283614A600361CE0280513033C031C95
:1001B000E528E5200730A100D030182103140800FD
:1001C0003614FE3C031989290517A60E361C361075
:1001D0008517F030850526080F3985048513A60E8E
:1001E0003618E728323017210314080084178004DA
:1001F000892983169B001C141A08892983169A00E2
:100200001C1555309D00AA309D009C149C18062991
:100210001C118929A301A200FF30A207031CA30718
:10022000031C89290330A100DF3018210C29A1010A
:10023000E83EA000A109FC30031C2129A0070318F7
:100240001E29A0076400A10F1E2920182729A01C21
:100250002B2900002B290800A20002303929A20016
:1002600003303929A20006303929A301A200043045
:100270003929A80023082102031D40292208200251
:10028000043003180130031902302805031DFF3024
:100290008929A2002008A6002408A0002608A4009E
:1002A0002108A6002508A1002608A5005929A501B6
:1002B000A4011030A600210DA40DA50D2208A40252
:1002C0002308031C230FA50203186D292208A40785
:1002D00023080318230FA5070310A00DA10DA60BDB
:1002E0005B29200889291030A800A101A001A70CD2
:1002F000A60C031C81292208A00723080318230F3A
:10030000A107A10CA00CA50CA40CA80B772924080C
:1003100089298313031383126400080083160615CA
:1003200006148615831207309F00831681018312FD
:100330000130CD0064000330A300E8300B21FE3013
:10034000A6200130A6205030A6204C30A6204C30EC
:10035000A6202D30A6205630A6203030A6202E30E4
:10036000A6203430A620FE30A620C030A62044307F
:10037000A6204C30A6203130A6204D30A620463095
:10038000A6204B30A6200730A300D0300B21003030
:10039000F920C6000130F920C7000230F920CB0057
:1003A0000630BA000230B8000630BB001030B90089
:1003B000C2303E2047083E2046083E20CE303C203A
:1003C0000630BA000830B800AC01FF30AA00AB011B
:1003D0000130AD004A080220CA000318942A0630F2
:1003E000BA000230B8000630BB001030B900C2308D
:1003F0003E2047083E2046083E20CE303E200030BA
:100400003C20F222A0230630BA000430B800AC0130
:10041000FF30AA000A30AB000130AD0048080220CE
:10042000C80003184D2A0630BA000130B800AC01EC
:10043000FF30AA000A30AB000130AD0049080220AD
:10044000C9000318602A0630BA000830B800AC01B1
:10045000FF30AA00AB010130AD004A080220CA00FB
:100460000318812A0630BA000230B8000630BB00FB
:100470001030B900C3303E202320CC00FE30A6202F
:10048000C730A62064004C1F472A4C30A6206400C9
:100490004C1B4C2A5830A620032A4D08C6070318C7
:1004A000C70A4608A0004708A1005D30A300C0307D
:1004B0003221031D5F2A9030C6000130C700EF29AA
:1004C0004608A0004708A1004D083521031D7C2ADD
:1004D0004608A0004708A1000130A30090302C215D
:1004E000031D772A4D08C602031CC703EA2BC03040
:1004F000C6005D30C700EA2B9030C6000130C7004F
:10050000EA2B640009304D020318902A4D08A6001A
:10051000A7010230A200A3017321CD00A023032A6A
:100520000130CD00A023032AFE30A6200130A620F2
:10053000FE30A6208030A6204D30A6207530A620A3
:100540006C30A6207430A6206930A6207030A6201A
:100550006C30A6203A30A620FE30A620C030A6205F
:100560004B0887200630BA000430B800AC01FF30D9
:10057000AA00AB010130AD0048080220C8000318F2
:10058000E02A0630BA000130B800AC01FF30AA0002
:10059000AB010130AD0049080220C9000318E92A67
:1005A0000630BA000830B800AC01FF30AA00AB0139
:1005B0000130AD004A080220CA000318EA2BB22A13
:1005C000CB0A640015304B02031CE82A0130CB0033
:1005D000942ACB03640001304B020318F12A143033
:1005E000CB00942A7D30A600A7014B08A200A301EE
:1005F0007321C4002508C5004608A6004708A700C7
:100600004408A2004508A3007321BC002508BD00D2
:100610000330A300E8304921C0002108C10046088A
:10062000A6004708A7004408A2004508A3007321BC
:10063000B2002508B3004608A6004708A7004408F2
:10064000A2004508A3007321B4002508B5003408B2
:10065000A0003508A100E830A2000330A300572114
:10066000B4002108B5003408A6003508A700E8301A
:10067000A2000330A3007321B4002508B50034089C
:100680003202C2003508031C013E3302C300420897
:10069000A6004308A7001930A200A3017321C200DD
:1006A0002508C3004208A0004308A100E830A200CA
:1006B0000330A3005721B2002108B3003208A6007E
:1006C0003308A700E830A2000330A3007321B20072
:1006D0002508B3003208C2023308031C013EC302DE
:1006E0004208A6004308A7000530A200A301732119
:1006F000C2002508C3004208A0004308A100E8305A
:10070000A2000330A3005721B2002108B300320831
:10071000A6003308A700E830A2000330A30073212D
:10072000B2002508B30032084202BE003308031CA1
:10073000013E4302BF003E08BE003F08BF00080064
:10074000FE30A6208030A6204108A5004008882061
:100750002E30A6203E08A0003F08A100A30164306F
:100760002F21031DC02B3030A6203E08A0003F08DB
:10077000A100A3010A302F21031DC02B3030A62079
:100780003F08A5003E088820FE30A620C030A620E5
:100790007D30A600A7014D08A200A3017321B2007D
:1007A0002508B3003208A6003308A7004B08A200B2
:1007B000A3017321B2002508B3003308A500320855
:1007C00088206B30A6204830A6207A30A620C8307A
:1007D0000A21080083169B0183124608FE20831617
:1007E00001309B0083124708FE20831602309B00D5
:0807F00083124B08FE20EF29E3
:02400E00703F01
:06420000C0004A000100AD
:00000001FF
